:1000000063280F39A00083161F088F3930389F00EE
:1000100083120310A00DA00D1F08C1392004013860
:100020009F000030A100323034209F149F18162802
:100030001E08A10083161E085E288316F838810565
:100040000F39810463000F3081045E28A301A200F0
:10005000FF30A207031CA307031C5E280330A10086
:10006000DF3034202828A101E83EA000A109FC309F
:10007000031C3D28A00703183A28A0076400A10F1D
:100080003A2820184328A01C4728000047280800C9
:10009000A20003304E28A20006304E28A8002308F4
:1000A0002102031D552822082002043003180130C4
:1000B000031902302805031DFF305E288313031344
:1000C00083126400080007309900850183161630FA
:1000D00085003E309F008312CC309F00C401C101D7
:1000E0000230C2000130C000BC01BD01FA30262040
:1000F00003300120BE002108BF0002300120BA00F9
:100100002108BB003E08A0003F08A1003B08A30057
:100110003A084B20031D96283A083E02BC003B08D3
:10012000031C013E3F02BD000130C3003E08A00099
:100130003F08A1003B08A3003A084820031DA92856
:100140003E083A02BC003F08031C013E3B02BD00D2
:10015000C30103300120BE002108BF00023001208E
:10016000BA002108BB0064004308013C031DBF28FE
:100170003C08BE023D08031C013EBF02C5283C08E6
:10018000BE073D080318013EBF0764000B30440260
:10019000031CCC280510851664000B304102031C9B
:1001A000D3288512051440083A07B2003B0803180B
:1001B000013EB3003E08A0003F08A1003308A300A1
:1001C00032084B20031DE828C40AC101A928FC28D5
:1001D00042083A02B2003B08031CFF3EB3003E084F
:1001E000A0003F08A1003308A30032084820031DE7
:1001F000FC28C10AC401A928C401C1010510851247
:0602000002301D20A928B8
:02400E00DC3F95
:00000001FF
